:020000040800F2
:100000000004022001020008D10E0008D50E0008ED
:10001000290F0008D50E0008FD0E00080302000895
:10002000030200080302000803020008D930000898
:10003000030200080302000803020008030200088C
:10004000030200080302000803020008030200087C
:100050000302000803020008313300085D33000882
:1000600089330008B5330008E133000803020008B3
:10007000030200080302000803020008030200084C
:10008000030200080302000803020008030200083C
:100090000302000803020008030200080D340008F0
:1000A000030200080302000803020008030200081C
:1000B000553100080302000803020008030200088B
:1000C00003020008030200080302000803020008FC
:1000D00003020008030200080302000803020008EC
:1000E0007534000803020008030200080302000838
:1000F00003020008030200080302000803020008CC
:1001000003020008030200080302000803020008BB
:1001100003020008030200080302000803020008AB
:10012000030200080302000803020008030200089B
:10013000030200080302000803020008030200088B
:10014000030200080302000803020008DD2700087C
:10015000030200080302000803020008030200086B
:10016000030200080302000803020008030200085B
:10017000030200080302000803020008030200084B
:10018000030200080302000803020008030200083B
:10019000030200080302000803020008030200082B
:1001A000030200080302000803020008030200081B
:1001B000030200080302000803020008030200080B
:1001C00003020008030200080302000803020008FB
:1001D00003020008030200080302000803020008EB
:1001E00003020008030200080302000803020008DB
:1001F00003020008030200080302000803020008CB
:1002000002E000F000F8FEE772B6394880F3088893
:10021000384880F3098838484EF60851CEF200017C
:10022000086040F20000CCF200004EF63471CEF2CD
:1002300000010860BFF34F8FBFF36F8F40F20000E3
:10024000C0F2F0004EF68851CEF200010860BFF314
:100250004F8FBFF36F8F4FF00000E1EE100A4EF6A4
:100260003C71CEF200010860062080F31488BFF3D1
:100270006F8F01F03BFF02F0B7FE4FF055301F4982
:100280001B4A91423CBF41F8040BFAE71C49194A4A
:1002900091423CBF41F8040BFAE71A491A4A1B4B3A
:1002A0009A423EBF51F8040B42F8040BF8E70020D5
:1002B0001749184A91423CBF41F8040BFAE701F094
:1002C00059FF02F0FBFE144C144DAC4203DA54F813
:1002D000041B8847F9E700F03FF8114C114DAC4280
:1002E00003DA54F8041B8847F9E701F041BF000026
:1002F0000004022000240220000000080000022068
:100300000004022098380008002402205024022013
:100310005024022058300220000200080002000889
:1003200000020008000200082DE9F04F2DED108AB0
:10033000C1F80CD0D0F80CD0BDEC108ABDE8F08F1D
:10034000002383F311882846A047002001F056FBC4
:1003500001F006FB00DFFEE770B5214C6FF01303E0
:1003600023700323002563706FF07F061E23A570A2
:10037000E57025716571A571E57125726672A372CC
:10038000E57200F009FD20B10E2325726672A3729A
:10039000E57201F06DFE044601F0A2FE0546D8B9F3
:1003A000104B9C421AD001339C4218BF054641F2C3
:1003B000883404BF01250024002001F063FE0DB144
:1003C00000F0B6F800F058FD00F038FC204600F0D0
:1003D0004FF900F0ADF8F9E70024EDE70446EBE74C
:1003E00050240220010007B008B500F0C9FBA0F1BD
:1003F00020035842584108BD07B5054B02211B8810
:10040000ADF8043001A800F009FC03B05DF804FB6E
:1004100058350008064991F8243033B100230822EA
:10042000086A81F8243000F02DBC0120704700BF1D
:10043000702402202DE9F84F234C94F8243005460F
:10044000884617468BBB2E46DFF87C90002F38D0AD
:1004500094F824A0BAF1000F05D12022FF214846CC
:10046000266200F0F7FCCAF10805BD4228BF3D46F0
:100470005FFA85FBAD0041462A4604EB8A0000F096
:10048000BFFC94F82430A7EB0B079B445FFA8BFB6F
:10049000BBF1080F2E44A844FFB284F824B0D5D194
:1004A000FFF7B8FF0028D1D108E0266A06EB8306E3
:1004B000B042C9D0FFF7AEFF0028C4D10020BDE88C
:1004C000F88F0120BDE8F88F7024022010B520239A
:1004D00083F311881248C3680BB101F015FB0023A8
:1004E000104A0F484FF47A7101F0D2FA002383F3D7
:1004F00011880D4C236813B12368013B23606368A6
:1005000013B16368013B6360084B1B7833B96368C0
:1005100023B9022000F06AFC3223636010BD00BFE3
:100520005C240220CD040008A0250220982402208B
:100530002DE9F041444B454953F8042F013201D1D4
:10054000BDE8F0818B42F7D1414C424B22689A4280
:1005500078D9414B9B6803F1006303F5C0339A429D
:1005600070D2002000F086FB3C4B0220187000F097
:1005700035FC3B4B1A6C00221A64196E1A66196E10
:10058000596C5A64596E5A66596E596941F0800126
:100590005961596921F0800159615969196941F01E
:1005A00000511961196921F0005119611B6972B676
:1005B0002C492D4B0B601D682468BFF34F8FBFF390
:1005C0006F8F2A4BC3F88420BFF34F8F5A6922F4F0
:1005D00080325A61BFF34F8FD3F88020C2F3C9062F
:1005E000C2F34E325201B70743F6E07E02EA0E082C
:1005F00038463146013948EA000CB1F1FF3FC3F8F3
:1006000074C200F14040F5D1203A12F1200FEDD133
:10061000BFF34F8FBFF36F8FBFF34F8FBFF36F8F5A
:100620005A6922F400325A610022C3F85022BFF303
:100630004F8FBFF36F8F202383F31188AD4685F36F
:1006400008882047BDE8F081FC7F01081C80010874
:1006500004800108FF7F0108502402209824022012
:100660000038024008ED00E00080010800ED00E0E5
:100670002DE9F04F99B0B34C01902022FF2110A832
:10068000A66800F0E7FBB04A1378A346A3B9AF48C9
:100690000121C3601170202383F31188C3680BB15B
:1006A00001F032FA0023AA4AA8484FF47A7101F007
:1006B000EFF9002383F31188019B13B1A54B019A35
:1006C0001A60A54AA349019F0292002313704B6050
:1006D00099461C461D469846012000F07FFB002FDE
:1006E00000F012829B4B1B68002B40F00D8219B06A
:1006F000BDE8F08F0220FFF777FE002840F0FB8175
:10070000019BB9F1000F08BF1F46944B1B88ADF841
:100710002C3002210BA800F081FADDE74FF47A704B
:1007200000F02EFA031E0393EADB0220FFF75CFEC3
:1007300082460028E4D0039B581E042800F2DD8185
:10074000DFE800F0030E1114170018A8052340F885
:10075000343D042100F062FA54464FF0000856E0A0
:1007600004217848F6E704217D48F3E704217D4819
:10077000F0E71C24204600F07FFA04340B9004219B
:100780000BA800F04BFA2C2CF4D1E5E7002DB7D0E4
:10079000002CB5D00220FFF727FE0546002800F008
:1007A000AF8101206C4C00F065FA0220207000F04F
:1007B00015FB4FF000095FFA89FA504600F06AFA1B
:1007C000074658B1504600F075FA09F101090028B2
:1007D000F1D12C46A9460027634B97E7012302205D
:1007E000237000F0F1FA3E46DBF808309E4206D254
:1007F000304600F041FA0130EBD10436F4E7029BB9
:1008000000261E70534BA9465E602C46374600F00A
:1008100029FB15B1002C18BF0027FFF7EDFD5BE7A2
:10082000002D3FF46DAF002C3FF46AAF029B022015
:10083000187000F0D3FA322000F0A2F9B0F1000AEB
:10084000C0F25E811AF0030540F05A81DBF80820FF
:1008500006EB0A03934200F25381BAF5807F00F25F
:100860004F8155450DDA4FF47A7000F089F9049004
:10087000049B002BC0F244813C4A049BAB540135DD
:10088000EFE7C820FFF7B0FD0546002800F03881EB
:100890001F2E11D8C6F12004544528BF544610AB72
:1008A00026F0030022463149184400F0A9FA2246F6
:1008B000FF212E4800F0CEFA4FEAAA0A5FFA8AF228
:1008C0002A493046FFF7B6FD0446002800F01A8199
:1008D00006EB8A0605469AE70220FFF785FD002809
:1008E0003FF40EAFFFF796FD00283FF409AF4FF03D
:1008F000000A5346DBF8082092451CD2BAF11F0FBC
:1009000012D8109A01320FD02AF0030218A90A4413
:1009100052F8202C0B92184604220BA900F018FB69
:100920000AF1040A0346E5E75046039300F0A4F9F0
:10093000039B0B90EFE718A8042140F84C3D00F012
:100940006DF964E7502402209C2502205C240220DB
:10095000CD040008A0250220982402205A35000862
:1009600054240220582402205C3500089C240220D4
:1009700018A8002340F8343D642100F02BF900282A
:100980007FF4BEAE0220FFF72FFD00283FF4B8AE83
:100990000B9800F0A1F918AB43F8480D0421184654
:1009A000CDE718A8002340F8343D642100F012F987
:1009B00000287FF4A5AE0220FFF716FD00283FF4C3
:1009C0009FAE0B9800F096F918AB43F8440DE5E79D
:1009D0000220FFF709FD00283FF492AE00F090F9E5
:1009E00018AB43F8400DD9E70220FFF7FDFC0028C3
:1009F0003FF486AE0BA9142000F088F9824618A8AF
:100A0000042140F83CAD00F009F951460BA896E7E7
:100A1000322000F0B5F8B0F1000AFFF671AE1AF01E
:100A2000030F7FF46DAEDBF808200AEB0803934256
:100A30003FF666AE0220FFF7D7FC00283FF460AE19
:100A40002AF0030AC244D0453FF4E1AE404600F02C
:100A500013F904210A900AA800F0E0F808F104084C
:100A6000F1E74FF47A70FFF7BFFC00283FF448AE7F
:100A7000FFF7D0FC00283FF4AFAE109B01330CD041
:100A8000082210A90020FFF7D5FC00283FF4A4AEEF
:100A90002022FF2110A800F0DDF9FFF7ADFC374858
:100AA00000F0B2FF23E6002D3FF42AAE002C3FF405
:100AB00027AE18A8002340F8343D642100F08AF8DE
:100AC000824600287FF41CAE0220FFF78DFC002830
:100AD0003FF416AE0390FFF78FFC41F2883000F030
:100AE00093FF0B9800F0F2F900F0BCF9039B574616
:100AF0001C461D46F0E5054689E64FF00008FFE577
:100B00002546FDE52C4667E6002000F039F8049004
:100B1000049B002BFFF6E3AD012000F055F9049B88
:100B2000213B122B3FF6D8AD01A252F823F000BFB3
:100B3000F50600081D0700088D070008D906000803
:100B4000D9060008D906000821080008110A000883
:100B5000D908000871090008A3090008D109000894
:100B6000D9060008E9090008D9060008630A000848
:100B70000F080008D9060008A70A0008A08601008F
:100B800037B5114B1A780132D2B20024012A01463E
:100B90008DF8074011D80D4803681D6A4FF47A7329
:100BA0004B4301220DF10701A847012805D1084B4D
:100BB0009DF807001C7003B030BD4FF4FA7000F0D0
:100BC00023FF4FF0FF30F6E70024022070260220BA
:100BD000AC25022038B50E4B1A780132D2B2012A68
:100BE00005460ED80B4803681C6A4FF47A734B43D2
:100BF00004222946A047042803D1074B002018707F
:100C000038BD4FF4FA7000F0FFFE4FF0FF3038BDF2
:100C10000024022070260220AC25022030B4054CAE
:100C20002368DD69044B0A46AC460146204630BCC9
:100C3000604700BF70260220A0860100F8B501F0D1
:100C40001BF9094C094E0A4F2070002530682378A3
:100C5000834207D901F00AF9336805440133BD42E4
:100C60003360F3D9F8BD00BFAD250220A8250220CE
:100C7000FF7F010001F0AEB900F1006000F5C03067
:100C80000068704700F10060920000F5C03001F08C
:100C900039B90000054B1A68054B1B789B1A834233
:100CA00002D9104401F0E2B800207047A8250220C4
:100CB000AD25022038B5074D04462868204401F0D0
:100CC000DDF828B928682044BDE8384001F0EEB8C6
:100CD00038BD00BFA825022010F0030308D1B0F5ED
:100CE000806F05D800F10050A0F5712000687047B2
:100CF00000207047014BC058704700BF20F4F01F20
:100D0000014B1868704700BF002004E0F0B5204B8D
:100D10001E68204B1F885D6893F90840C6F30B02DC
:100D2000BA424FEA164622D09F89BA4221D01F8B81
:100D3000BA4206D102220C2404FB02335D6893F907
:100D40000840B6F5805F16D041F201039E4208BF0D
:100D50005A24421E0A44013D0B46934215D215F90E
:100D6000016F581C4EB1034600F8016CF5E70022F4
:100D7000E1E70122DFE74124EBE72C2582421D70E9
:100D800001D9981C5C70401AF0BD1846FBE700BF03
:100D9000002004E004240220094B5B88B3F5805F47
:100DA00009D041F20102934207D10122054B03EB26
:100DB0008203D87870470022F8E70020704700BF10
:100DC000002004E060350008022802BF024B4FF407
:100DD00080329A61704700BF00100240022802BFB3
:100DE000014B01229A61704700100240022801BFA6
:100DF000024A536983F001035361704700100240B7
:100E000010B50023934203D0CC5CC4540133F9E7FE
:100E100010BD000030B5441E14F9010F0B4660B13F
:100E200093F90050854201F1010106D11AB993F9F5
:100E30000020801A30BD013AEEE7002AF7D11046B3
:100E400030BD000002460346981A13F9011B002921
:100E5000FAD1704702440346934202D003F8011BC3
:100E6000FAE77047024B1A78024B1A70704700BFBE
:100E7000AC2502200024022038B5104D104C284625
:100E800000F002F92146284600F02AF924680D48AE
:100E9000E26ED2F8043843F00203C2F8043800F0DE
:100EA000B3FD0949204600F029FAE26ED2F8043871
:100EB00023F00203C2F8043838BD00BF70260220B8
:100EC0001036000840420F00383600087047000016
:100ED000FEE7000000B59BB0EFF309816822684689
:100EE000FFF78EFFEFF30583034B9A6B9A6A9A6ABA
:100EF0009A6A9A6A9B6AFEE700ED00E000B59BB033
:100F0000EFF3098168226846FFF77AFFEFF3058364
:100F1000044B9A6B9A6A9A6A9A6A9A6A9A6A9B6A64
:100F2000FEE700BF00ED00E000B59BB0EFF30981E4
:100F300068226846FFF764FFEFF30583034B5A6BA3
:100F40009A6A9A6A9A6A9A6A9B6AFEE700ED00E0DA
:100F500030B5084D0A4491420BD011F8013B0924E9
:100F60005840013CF7D040F300032B4083EA500087
:100F7000F7E730BD2083B8ED002304491A465A50E4
:100F8000C8180833802B4260F9D17047B025022081
:100F9000026843681143016003B1184770470000BD
:100FA00013B5446BD4F894341A681178042915D118
:100FB000217C022912D11979128901238B40134215
:100FC0000CD101A904F14C0001F082FED4F8944444
:100FD000019B21790246206800F0E0F902B010BDC3
:100FE000143001F005BE00004FF0FF33143001F063
:100FF000FFBD00004C3001F0D7BE00004FF0FF33C2
:101000004C3001F0D1BE0000143001F0D3BD00001F
:101010004FF0FF31143001F0CDBD00004C3001F035
:10102000A3BE00004FF0FF324C3001F09DBE000027
:10103000D0F8942438B5136819780429054601D0EE
:10104000012038BD017C0229FAD112795C89012086
:1010500090400440F4D105F1140001F065FD024612
:101060000028EDD0D5F894544FF48073286869793E
:1010700000F082F9204638BD406BFFF7D9BF000071
:1010800000207047704700007FB5124B03600023BB
:1010900043608360C360012502260F4B057404463C
:1010A0000290019300F18402294600964FF4807368
:1010B000143001F015FD094B0193029400964FF492
:1010C000807304F52372294604F14C0001F0DCFD25
:1010D00004B070BD9435000879100008A10F000815
:1010E0000B68202282F311880A7903EB82021062D6
:1010F0004A790D3243F822008A7912B103EB820358
:10110000186202230374C0F89414002383F3118837
:101110007047000038B5037F044613B190F854308F
:10112000ABB9201D01250221FFF732FF04F11400A5
:1011300025776FF0010100F08FFC84F8545004F122
:101140004C006FF00101BDE8384000F085BC38BDAF
:1011500010B5012104460430FFF71AFF002323775E
:1011600084F8543010BD000038B504460025143012
:1011700001F0CEFC04F14C00257701F09DFD201D0F
:1011800084F854500121FFF703FF2046BDE83840A2
:10119000FFF74EBF90F85C3003F06003202B19D1AD
:1011A00090F85D20212A0AD0222A4FF000030ED0A9
:1011B000202A0FD1084A02650722426504E0064B47
:1011C000036507234365002383650120704703659A
:1011D0004365F9E70020704728240220D0F89434B2
:1011E00037B51A681178042904461AD1017C0229FE
:1011F00017D11979128901238B40134211D100F1C3
:101200004C05284601F018FE58B101A9284601F006
:101210005FFDD4F89444019B21790246206800F0D8
:10122000BDF803B030BD000000EB8103F7B51C6AC8
:1012300005460E46F4B1202383F3118805EB86079B
:10124000201D0821FFF7A4FEFB685B691B684C3476
:1012500013B1204601F04AFD01A9204601F038FDF6
:10126000024648B1019B3146284600F097F800231A
:1012700083F3118803B0F0BDFB685A691268002A35
:10128000F5D01B8A013B1340F1D105F15C02EAE77E
:101290000D3138B550F82140DCB1202383F311889B
:1012A000D4F894241368527903EB8203DB689B69BA
:1012B0005D6845B104216018FFF76AFE294604F114
:1012C000140001F03BFC2046FFF7B2FE002383F33D
:1012D000118838BD7047000000F0D2BF01230370B1
:1012E0000023436000F1240200F1380142F8043B7E
:1012F0008A421361FAD103814381704738B50446AD
:10130000202383F3118800254160C5600561456194
:101310008561C561056200F0C3FF0223237085F378
:10132000118838BD70B500EB810305465069DA605D
:101330000E46144618B110220021FFF78BFDA0695C
:1013400018B110220021FFF785FD31462846BDE87F
:10135000704001F06FB80000028902F001020281C2
:10136000428902F0010242810022026142618261EF
:10137000C261026201F0F2B8F0B400EB8104478967
:10138000E4680125A4698D403D4345812360002325
:10139000A2606360F0BC01F00DB90000F0B400EB96
:1013A00081040789E468012564698D403D43058116
:1013B00023600023A2606360F0BC01F087B90000E5
:1013C00070B50223002504460370A0F8645080F82D
:1013D000665080F8675005814581C56005614561AB
:1013E0008561C561056280F84C5000F0BFFF6368FD
:1013F0001B6823B129462046BDE87040184770BDE0
:10140000436802781B6880F86820052202700BB1DF
:101410000421184770470000436890F868201B6853
:1014200002700BB1052118477047000090F84C304E
:1014300070B5044613B1002380F84C3004F15C020F
:10144000204601F0ADF863689B6863BB94F85C507C
:1014500015F0600615D194F85D3005F07F0545EA7A
:10146000032540F202339D4200F00E815BD8022D2D
:1014700000F0DC803FD8002D00F08780012D00F0C7
:10148000CF800021204601F0F7FA0021204601F02C
:10149000E9FA63681B6813B10621204698470623C2
:1014A00084F84C3070BD204698470028CED094F880
:1014B000632094F8623043EA0223626D934238BF9E
:1014C000636594F95C30656D002B4FF0200380F26A
:1014D000FD80002D00F0EC80092284F84C2083F37D
:1014E00011880021636D226D2046FFF757FF00230E
:1014F00083F3118870BDB5F5817F00F0B180B5F53B
:10150000407F49D0B5F5807FBBD194F85E30012B88
:10151000B7D1B4F8643023F00203A4F86430266530
:101520006665A665C3E740F201639D421ED8B5F526
:10153000C06F3BD2B5F5A06FA3D1B4F85C30B3F562
:10154000A06F0ED194F85E3084F86630204600F02B
:1015500065FF63681B6813B1012120469847032388
:101560002370002323656365A365A0E7B5F5106FBD
:1015700032D040F602439D4252D0B5F5006F80D183
:1015800004F167032365012324E004F16403236568
:1015900002236365A5658AE794F85E30012B7FF42A
:1015A00070AFB4F8643043F00203B6E794F86120FA
:1015B000616894F860304D6894F85F1043EA022344
:1015C000204694F85E20A84700283FF45AAF4368AD
:1015D000236503686365A4E72378042B10D12023D7
:1015E00083F311882046FFF7B7FE86F311886368FE
:1015F00084F867601B68032121700BB1204698476F
:1016000094F85E30002BACD084F86730042323704C
:1016100063681B68002BA4D0022120469847A0E7EE
:10162000374B23650223636500239DE794F8601020
:1016300011F0800F204601F00F010ED000F0A2FF44
:10164000012806D002287FF41CAF2E4B236560656D
:1016500067E72D4B2365656563E700F085FFEFE7DE
:1016600094F85E30002B7FF40CAF94F8603013F0E8
:101670000F013FF476AF1A06204602D501F010FAAA
:101680006FE701F003FA6CE794F85E30002B7FF40B
:10169000F8AE94F8603013F00F013FF462AF1B0610
:1016A000204602D501F0E8F95BE701F0DBF958E7E5
:1016B000142284F84C2083F311882B462A462946AD
:1016C0002046FFF759FE85F3118870BD5DB11522E4
:1016D00084F84C2083F311880021636D226D20462D
:1016E000FFF74AFE03E70B2284F84C2083F31188AE
:1016F0002B462A4629462046FFF750FEE3E700BF67
:10170000C4350008BC350008C035000838B590F86D
:101710004C300446152B29D8DFE803F03E28282852
:1017200028283E28280B293928282828282828282E
:101730003E3E90F8631090F86220436D42EA012229
:101740009A4214D9C268128AB3FBF2F502FB15352E
:101750006DB9202383F311882B462A462946FFF7CB
:101760001DFE85F311880A2384F84C3038BD1423FC
:1017700084F84C30202383F3118800231A4619463D
:101780002046FFF7F9FD002383F3118838BD836DF0
:1017900003B198470023E7E7002101F06DF900212C
:1017A000204601F05FF963681B6813B106212046EB
:1017B00098470623D8E7000090F84C20152A38B542
:1017C000044622D80123934040F6416213421DD1C2
:1017D00013F480150FD19B0217D50B2380F84C30E2
:1017E000202383F311882B462A462946FFF7D6FD8E
:1017F00085F3118838BDC3689B695B682BB9836D1D
:1018000003B19847002384F84C3038BD002101F023
:1018100033F90021204601F025F963681B6813B1F4
:101820000621204698470623EDE70000024B0022E0
:101830001B605B609A6070473026022000230374AF
:101840008268054B1B6899689142FBD25A68036015
:1018500042601060586070473026022008B520238F
:1018600083F31188037C032B05D0042B0DD02BB9F7
:1018700083F3118808BD436900221A604FF0FF33DB
:101880004361FFF7DBFF0023F2E790E80C001A60EA
:1018900002685360F2E70000002303748268054B7E
:1018A0001B6899689142FBD85A68036042601060D7
:1018B0005860704730260220054B19690874186873
:1018C00002681A605360186101230374FEF72CBD8F
:1018D0003026022030B54B1C87B005460A4C10D08C
:1018E00023690A4A01A800F0D3F82846FFF7E4FF6D
:1018F000049B13B101A800F007F92369586907B0E8
:1019000030BDFFF7D9FFF8E7302602205D18000848
:1019100038B50C4D41612B6981689A689142044643
:1019200003D8BDE83840FFF789BF1846FFF786FFA8
:1019300001232C61014623742046BDE83840FEF7A0
:10194000F3BC00BF30260220044B1A681B69906864
:101950009B68984294BF00200120704730260220E7
:1019600010B5084C236820691A682260546001226F
:1019700023611A74FFF790FF01462069BDE810400B
:10198000FEF7D2BC302602208260022202740022BE
:10199000427470478368A3F17C0243F80C2C0269FF
:1019A00043F83C2C426943F8382C074A43F81C2C76
:1019B000C26843F8102C022203F8082C002203F816
:1019C000072CA3F1180070474103000810B520232D
:1019D00083F31188FFF7DEFF00210446FFF798FF2D
:1019E000002383F31188204610BD0000024B1B69C1
:1019F00058610F20FFF760BF30260220202383F3B9
:101A00001188FFF7F3BF000008B50146202383F3D8
:101A100011880820FFF75EFF002383F3118808BDBB
:101A200049B1064B42681B6918605A6013604360F5
:101A30000420FFF74FBF4FF0FF30704730260220E1
:101A40000368984206D01A680260506059611846CF
:101A5000FFF7F4BE7047000038B504460D46206815
:101A6000844200D138BD036823605C604561FFF7A4
:101A7000E5FEF4E7054B03F114025A619A614FF059
:101A8000FF32DA6100221A62704700BF302602205E
:101A9000F8B503614FF08043C2605C6A194B1A4687
:101AA000022952F8145F38BF0221954206461F46AC
:101AB0000AD1586198611C6205604560816008190F
:101AC000BDE8F84001F0DAB9186AAB68241A0C19BD
:101AD00002D3E41A2D6804E09C4202D2204401F0B3
:101AE000DBF9AB689C42F4D86B68736035601E60AC
:101AF0006E60B460A9684FF0FF33091BA960FB61F9
:101B0000F8BD00BF3026022010B41B4C234653F80A
:101B1000141F814210D0416802680A600268516057
:101B20009A424FF00001C16003D0936881680B4472
:101B300093605DF8044B70470A68626100209A4226
:101B40005360C86003D15DF8044B01F09FB99368FE
:101B50008868034493604FF08042206A526A121AE8
:101B60009342E6D9991A012998BF931C18445DF84D
:101B7000044B01F091B900BF3026022000207047CD
:101B8000FEE70000704700004FF0FF307047000094
:101B9000022906D0032906D00129064818BF0020D3
:101BA000704705487047032A9ABF044800EBC200FB
:101BB0000020704794360008483600083024022080
:101BC00070B59AB001AD064608462946144600F0A5
:101BD00095F82846FFF736F9C0B2431C5B0086E84B
:101BE0001800237003236370002302341946DAB20D
:101BF000904204F1020401D81AB070BDEA5C04F806
:101C0000022C04F8011C0133F1E7000008B5202381
:101C100083F311880348FFF7E1FA002383F3118867
:101C200008BD00BF7026022010B50446052916D84D
:101C3000DFE801F016150316161D202383F3118823
:101C40000E4A0121FFF76EFB20460D4A0221FFF7E5
:101C500069FB0C48FFF788FA002383F3118810BD55
:101C6000202383F311880748FFF754FAF4E7202371
:101C700083F311880348FFF76BFAEDE7C8350008D6
:101C8000EC3500087026022038B50C4D0C4C0D497F
:101C90002A4604F10800FFF793FF05F1CA0204F198
:101CA00010000949FFF78CFF05F5CA7204F118000E
:101CB0000649BDE83840FFF783BF00BF382B02203C
:101CC0003024022018360008223600082D3600087D
:101CD00070B5044608460D46FFF7B4F8C6B2204674
:101CE000013403780BB9184670BD32462946FFF718
:101CF00091F80028F3D1012070BD00002DE9F84FC4
:101D000005460C46FFF79EF82A49C6B22846FFF75B
:101D1000DFFF29492846FFF7DBFF08B11036F6B28E
:101D2000632E0DD8DFF88C80DFF88C90234FDFF81E
:101D300094A0DFF894B02E7846B92670BDE8F88FED
:101D400029462046BDE8F84F01F0FEBB252E2CD1D8
:101D5000072241462846FFF75DF858B9DBF8003006
:101D60002360BBF80430A3809BF80630A3710735CD
:101D70000734E0E7082249462846FFF74BF8A0B9A8
:101D80000F4BA21C13F8011F09095345C95D02F846
:101D9000021C197801F00F0102F10202C95D02F87C
:101DA000031CEFD118340835C5E72670013501341E
:101DB000C1E700BFB43600082D360008C43600085D
:101DC0001FF4F01F2BF4F01FBC360008BFF34F8F39
:101DD000024AD368DB03FCD4704700BF003C0240DA
:101DE00008B5074B1B7853B9FFF7F0FF054B1A698D
:101DF000002ABFBF044A5A6002F188325A6008BD07
:101E0000962D0220003C02402301674508B5054B92
:101E10001B7833B9FFF7DAFF034A136943F0004335
:101E2000136108BD962D0220003C02400B2870B5BE
:101E300013D80B4A0B4C137863B90B4E4FF000616B
:101E400044F8231056F8235001330C2B2944F7D1C2
:101E50000123137054F8200070BD002070BD00BF36
:101E6000C82D0220982D0220D8360008014B53F8C7
:101E700020007047D83600080C2070470B2810B59A
:101E8000044601D9002010BDFFF7D0FF064B53F8E0
:101E900024301844C21A0BB9012010BD1268013257
:101EA000F0D1043BF6E700BFD83600080B2810B588
:101EB000044621D8FFF78AFFFFF792FF0F4AF3236A
:101EC000D360C300DBB243F4007343F00203136139
:101ED000136943F480331361FFF778FFFFF7A6FF20
:101EE000074B53F8241000F0DDF8FFF78FFF204672
:101EF000BDE81040FFF7C2BF002010BD003C02400B
:101F0000D83600082DE9F84312F00103154640D1F8
:101F10008218B2F1026F3CD22C4B1B6813F0010304
:101F200037D02B4CFFF75CFFF323E360FFF74EFF46
:101F300040F20127032D01D9830713D0244C0F460B
:101F4000401A40F20118EB1B0B44012B00EB070673
:101F5000236924D823F001032361FFF757FF0120F1
:101F6000BDE8F883236923F44073236123693B436D
:101F7000236151F8046B0660BFF34F8FFFF726FF14
:101F800003689E4208D0236923F001032361FFF711
:101F90003DFF0020BDE8F883043D0430CAE723F488
:101FA00040732361236943EA08032361B94637F884
:101FB000023B3380BFF34F8FFFF708FF3688B9F835
:101FC0000030B6B2B342BED0DDE700BF00380240F9
:101FD000003C0240084908B50B7828B153B9FFF717
:101FE000FFFE01230B7008BD23B1BDE80840087057
:101FF000FFF70CBF08BD00BF962D022010B50244AC
:10200000064B0439D2B2904200D110BD441C00B23C
:1020100053F8200041F8040FE0B2F4E750280040E4
:10202000104B30B51C6F240407D41C6F44F40074AB
:102030001C671C6F44F400441C670B4C236843F47A
:10204000807323600244094B0439D2B2904200D11C
:1020500030BD441C00B251F8045F43F82050E0B298
:10206000F4E700BF003802400070004050280040F4
:1020700007B5012201A90020FFF7C0FF019803B0B6
:102080005DF804FB13B50446FFF7F2FFA04206D04B
:1020900002A9012241F8044D0020FFF7C1FF02B060
:1020A00010BD00000144BFF34F8F064B884204D39C
:1020B000BFF34F8FBFF36F8F7047C3F85C022030C0
:1020C000F4E700BF00ED00E0034B1B689B0042BF3C
:1020D000024B01221A70704774380240C92D022049
:1020E000014B1878704700BFC92D0220F0B5BFF32F
:1020F0004F8FBFF36F8F1D4B0021C3F85012BFF3FA
:102100004F8FBFF36F8F5A6942F400325A61BFF3A9
:102110004F8FBFF36F8FC3F88410BFF34F8FD3F887
:102120008020C2F3C904C2F34E325201A50743F620
:10213000E07602EA060E284621464EEA00070139FB
:10214000C3F860724F1C00F14040F6D1203A12F102
:10215000200FEED1BFF34F8F5A6942F480325A619B
:10216000BFF34F8FBFF36F8FF0BD00BF00ED00E0F6
:10217000FEE70000084A094B09498B4204D3094A8B
:102180000021934205D3704752F8040F43F8040B23
:10219000F3E743F8041BF4E7E43800085830022062
:1021A0005830022058300220036F30B500229D685D
:1021B000C46E11464FF0FF3004EB421301329542DA
:1021C000C3F80019C3F81019C3F80809C3F8001BB5
:1021D000C3F8101BC3F8080BEED24FF00113C4F87C
:1021E0001C3830BD890141F02001016103699B0663
:1021F000FCD4122000F0DEBE204B03EB80022DE960
:10220000F047D2F80CE0DD6EDEF81420461CD2F860
:1022100000C005EB063605EB4018516861450BD34D
:10222000D5F83428012303FA00F022EA0000C5F8AB
:1022300034081846BDE8F087BEF81040ACEB010347
:10224000A34228BF2346D8F81849A4B2B3EB840FA1
:1022500010D894681F46A4F1040959F804AFC6F8D1
:1022600000A0042F01D9043FF7E71C440B449460FD
:102270005360D2E70020BDE8F08700BFCC2D0220DC
:1022800010B5054C2046FFF729F84FF0A043E36650
:10229000024B236710BD00BFCC2D02202C37000855
:1022A0000378012B70B5054650D12A4BC46E984275
:1022B0001BD1294B5A6B42F080025A635A6D42F08F
:1022C00080025A655A6D5A6942F080025A615A6911
:1022D00022F080025A610E2143205B6900F0EAFB84
:1022E0001E4BE3601E4BC4F800380023C4F8003EC8
:1022F000C0232360EE6E4FF40413A3633369002BF5
:10230000FCDA012333610C2000F054FE3369DB0753
:10231000FCD4122000F04EFE3369002BFCDA0026BC
:10232000A6602846FFF740FF6B68C4F81068DB68BA
:10233000C4F81468C4F81C684BB90A4BA3614FF089
:10234000FF336361A36843F00103A36070BD064BD4
:10235000F4E700BFCC2D02200038024040140040BA
:1023600003002002003C30C0083C30C0F8B5C46E09
:10237000054600212046FFF735FF296F00234FF067
:1023800001128F68C4F834384FF00066C4F81C2876
:102390004FF0FF3004EB431201339F42C2F8006953
:1023A000C2F8006BC2F80809C2F8080BF2D20B6839
:1023B000EA6E6B67636210231361166916F01006EC
:1023C000FBD1122000F0F6FDD4F8003823F4FE63B0
:1023D000C4F80038A36943F4402343F01003A36119
:1023E0000923C4F81038C4F814380A4BEB604FF0D6
:1023F000C043C4F8103B084BC4F8003BC4F8106954
:10240000C4F800396B6F03F1100243F480136A675C
:10241000A362F8BD0837000840800010C26E90F833
:102420006610D2F8003823F4FE6343EA0113C2F8C1
:10243000003870472DE9F0410EB200EB86080D46DA
:10244000D8F80C100F6807F00303022B50D0032BB1
:1024500050D03D4A3D4F012B18BF1746C46E4FEA7E
:10246000451E04EB0E030022C3F8102B8A6905F108
:10247000100C002A40D04A8A05F158035B013A4308
:10248000E2500123D4F81C2803FA0CF31343A644AA
:102490004A69C4F81C380023CEF8103905F13F030F
:1024A000002A39D00A8A898B9208012988BF4A43B9
:1024B000416F04EB8303561841EA024246672946FE
:1024C0005A602046FFF78EFED8F80C301B8A43EA8C
:1024D00085531F4305F148035B01E7500123D4F8FE
:1024E0001C2803FA05F51543C4F81C58BDE8F08113
:1024F000174FB3E7174FB1E704EB4613D3F8002BA0
:1025000022F40042C3F8002BD4F81C28012303FA5C
:102510000CF322EA0303BAE704EB83030E4A5A6082
:1025200004EB461629462046FFF75CFED6F8003934
:1025300023F40043C6F80039D4F81C38012202FA0B
:1025400005F523EA0505CFE70080001000800410A0
:102550000080081000800C1000040002026F126856
:102560004267FFF721BE00005831C36E49015B5836
:1025700013F4004004D013F4001F14BF0120022004
:10258000704700004831C36E49015B5813F40040A6
:1025900004D013F4001F14BF012002207047000074
:1025A00000EB8101CB68196A0B6813604B685360BC
:1025B0007047000000EB810330B5DD68AA6913683D
:1025C000D36019B9402B84BF402313606B8A146811
:1025D000C26E1C44013CB4FBF3F46343033323F0A9
:1025E000030302EB411043EAC44343F0C043C0F885
:1025F000103B2B6803F00303012B09B20ED1D2F874
:10260000083802EB411013F4807FD0F8003B14BF70
:1026100043F0805343F00053C0F8003B02EB4112FB
:10262000D2F8003B43F00443C2F8003B30BD000049
:102630002DE9F041244DEE6E06EB40130446D3F82D
:10264000087BC3F8087B38070AD5D6F81438190771
:1026500006D505EB84032146DB6828465B6898476E
:10266000FA072FD5D6F81438DB072BD505EB8403F2
:10267000D968CCB98B69488A5E68B6FBF0F200FB7A
:1026800012628AB91868DA6890420DD2121A83E889
:102690001400202383F311880B482146FFF78AFF9B
:1026A00084F31188BDE8F081012303FA04F26B89F9
:1026B00023EA02036B81CB6823B121460248BDE8BF
:1026C000F0411847BDE8F081CC2D022000EB8103DA
:1026D00070B5DD68C36E6C692668E6604A0156BB5A
:1026E0001A444FF40020C2F810092A6802F00302CD
:1026F000012A0AB20ED1D3F8080803EB421410F4F1
:10270000807FD4F8000914BF40F0805040F00050A2
:10271000C4F8000903EB4212D2F8000940F004406B
:10272000C2F80009D3F83408012202FA01F101438A
:10273000C3F8341870BD19B9402E84BF4020206002
:1027400020682E8A841940F00050013C1A44B4FBE2
:10275000F6F440EAC440C6E7F8B504461E48C56E24
:1027600005EB4413D3F80869C3F80869F10717D5D6
:10277000D5F81038DA0713D500EB8403D9684B6914
:102780001F68DA68974218D2D21B00271A605F6070
:10279000202383F311882146FFF798FF87F31188E0
:1027A000330617D5D5F834280123A340134211D09E
:1027B0002046BDE8F840FFF71FBD012303FA04F2ED
:1027C000038923EA020303818B68002BE8D02146AA
:1027D0009847E5E7F8BD00BFCC2D0220A0482DE9C1
:1027E000F84FC56E6E69AB691E4016F4805F6E616E
:1027F000044605D0FEF7E4FDBDE8F84F00F07CBCD0
:10280000002E12DAD5F8003E95489B071EBFD5F87A
:10281000003E23F00303C5F8003ED5F8043823F04A
:102820000103C5F80438FEF7F7FD370502D58C48DB
:10283000FEF7E6FDB0040CD5D5F8083813F0060F06
:10284000EB6823F470530CBF43F4105343F4A053CC
:10285000EB60310704D56368DB680BB180489847AB
:10286000F2026FD4B3020CD5D4F86C80DFF8F0A17B
:1028700000274FF00109236F9B68F9B28B4280F06B
:102880009C80F70619D5E16E0A6AC2F30A1702F0B6
:102890000F0302F4F012B2F5802F00F0B680B2F50B
:1028A000402F0AD104EB830301F58051DB68186ADD
:1028B00000231A469F4240F09C803303D5F8184805
:1028C0001DD5E70302D50020FFF7B2FEA50302D510
:1028D0000120FFF7ADFE600302D50220FFF7A8FE3E
:1028E000210302D50320FFF7A3FEE20202D5042054
:1028F000FFF79EFEA30202D50520FFF799FE77039E
:102900007FF57AAFE60702D50020FFF725FFA50780
:1029100002D50120FFF720FF600702D50220FFF754
:102920001BFF210702D50320FFF716FFE20602D5A1
:102930000420FFF711FFA3067FF55EAF0520FFF728
:102940000BFF59E7D4F86C80DFF814A100274FF093
:102950000109236F9B685FFA87FB5B4582D308EB15
:102960004B13D3F8002902F44022B2F5802F22D174
:10297000D3F80029002A1EDAD3F8002942F0904249
:10298000C3F80029D3F80029002AFBDB5946E06E82
:10299000FFF728FC228909FA0BF322EA03032381BB
:1029A00004EB8B03DB689B6813B15946504698478C
:1029B0005846FFF721FC0137CBE708EB4112D2F86C
:1029C000003B03F44023B3F5802F10D1D2F8003B35
:1029D000002B0CDA628909FA01F322EA030363810E
:1029E00004EB8103DB68DB680BB150469847013785
:1029F00041E79C0708BF0A68072B98BF027003F1E4
:102A000001039CBF120A013054E7023304EB830236
:102A100001F58051526890690268D0F808C040689A
:102A2000A2EB000E0022104697420AD104EB830469
:102A300063689B699A683A449A605A6817445F6071
:102A40003BE712F0030F08BF0868964588BF8CF873
:102A5000000002F1010284BF000A0CF1010CE3E75F
:102A6000CC2D0220C36E03EB4111D1F8003B43F49F
:102A70000013C1F8003B7047C36E03EB4111D1F85E
:102A8000003943F40013C1F800397047C36E03EBFB
:102A90004111D1F8003B23F40013C1F8003B70470B
:102AA000C36E03EB4111D1F8003923F40013C1F8D0
:102AB0000039704700F1604300F01F02400903F540
:102AC000614309018000C9B200F1604083F800133E
:102AD00000F5614001239340C0F8803103607047E6
:102AE00030B5039C0172043304FB0325C361049BCE
:102AF00003630021059B00604060C1604261026188
:102B00008561046242628162C162436330BD00003C
:102B10000022416A41610161C2608262C2626FF05B
:102B20000101FEF799BF000003694269934203D196
:102B3000C2680AB100207047181D70470369196008
:102B4000C2680132C260C269134482690361934260
:102B500024BF436A03610021FEF772BF38B5044603
:102B60000D46E3683BB16269131D1268A36213440A
:102B7000E362002038BD237A33B929462046FEF7A8
:102B80004FFF0028EDDA38BD6FF00100FBE70000D1
:102B9000C368C269013BC3604369134482694361EE
:102BA000934224BF436A436100238362036B03B1F2
:102BB0001847704770B52023044683F31188866A4E
:102BC0003EB9FFF7CBFF054618B186F311882846BA
:102BD00070BDA36AE26A13F8015BA362934202D359
:102BE0002046FFF7D5FF002383F31188EFE70000AD
:102BF0002DE9F84F04460E4690469946202787F364
:102C000011880025AA46D4F828B0BBF1000F09D1DD
:102C100049462046FFF7A2FF20B18BF311882846D2
:102C2000BDE8F88FA16AE36AA8EB050B5B1A9B4528
:102C300028BF9B46BBF1400F1BD9334601F1400230
:102C400051F8040B43F8040B9142F9D1A36A4033C5
:102C50004036A3624035A26AE36A9A4202D3204614
:102C6000FFF796FF8AF311884545D8D287F311887C
:102C7000C9E730465A46FEF7C3F8A36A5B445E4490
:102C8000A3625D44E7E7000010B5029C01720433C3
:102C900003FB0421C36100238362C362039B0363BC
:102CA000049B00604060C460426102618161046213
:102CB0004262436310BD0000026AC260426A426120
:102CC000026100228262C2626FF00101FEF7C4BE9F
:102CD000436902699A4203D1C2680AB10020704771
:102CE000184650F8043B0B6070470000C368C26987
:102CF0000133C3604369134482694361934224BF33
:102D0000436A43610021FEF79BBE000038B50446CC
:102D10000D46E3683BB123691A1DA262E2691344C0
:102D2000E362002038BD237A33B929462046FEF7F6
:102D300077FE0028EDDA38BD6FF00100FBE70000F8
:102D400003691960C268013AC260C26913448269AA
:102D50000361934224BF436A036100238362036BD0
:102D600003B118477047000070B5202304460E4693
:102D700083F31188856A35B91146FFF7C7FF10B193
:102D800085F3118870BDA36A1E70A36AE26A0133DD
:102D90009342A36204D3E16920460439FFF7D0FFD0
:102DA000002080F3118870BD2DE9F84F04460D46D0
:102DB00091469A464FF0200888F311880026B346C2
:102DC000A76A4FB951462046FFF7A0FF20B187F30D
:102DD00011883046BDE8F88FA06AE76AA9EB0603C0
:102DE0003F1A9F4228BF1F46402F1BD905F14003C1
:102DF00055F8042B40F8042B9D42F9D1A36A4033C7
:102E0000A3624036A26AE36A9A4204D3E16920468B
:102E10000439FFF795FF8BF311884E45D9D288F31B
:102E20001188CDE729463A46FDF7EAFFA36A3B44FD
:102E30003D44A3623E44E5E7026943699A4203D1F7
:102E4000C3681BB9184670470023FBE7836A002B51
:102E5000F8D0043B9B1AF5D01360C368013BC360F4
:102E6000C3691A44836902619A4224BF436A0361B9
:102E7000002383620123E5E700F080B94FF080432F
:102E8000002258631A610222DA6070474FF08043D3
:102E90000022DA60704700004FF0804358637047AB
:102EA000FEE7000010B5194CFEF7C0FCFEF7E2FD8E
:102EB000802217492046FEF767FD012344F8180CCD
:102EC0000374144B144AD96821F4E0610904090C15
:102ED0000A431249DA60CA6842F08072CA60104A36
:102EE0001049C2F8B01F116841F0010111601022B1
:102EF000DA77202283F82220002383F3118862B638
:102F00000948BDE81040FEF761BD00BF5826022009
:102F10003837000800ED00E00003FA05F0ED00E0AE
:102F2000001000E055CEACC5403700082DE9F84F41
:102F30001F4C4FF00008656904F11407C1464FF0BB
:102F40008043266A5B6AAA689E1B96421DD34FF097
:102F5000200AAA68236AD5F80CB0134423622B68B0
:102F6000BB425F60A6EB02066361C5F80C8001D12D
:102F7000FFF78CFF89F311882869D8478AF31188F5
:102F80006569AB689E42E4D2D9E76269BA420CD067
:102F9000916823628E1B9660A86802282CBF1818BF
:102FA000981CBDE8F84FFFF777BFBDE8F88F00BF6A
:102FB00030260220034B59685A68521A9042FBD8B7
:102FC000704700BF001000E04B6843608B6883606F
:102FD000CB68C3600B6943614B6903628B694362D1
:102FE0000B6803607047000008B5274B27481A6933
:102FF00040F2FF710A431A611A6922F4FF6222F05B
:1030000007021A611A691A6B0A431A631A6D0A4396
:103010001A651F4A1B6D1146FFF7D6FF1D4802F1C6
:103020001C01FFF7D1FF1C4802F13801FFF7CCFF6C
:103030001A4802F15401FFF7C7FF194802F1700165
:10304000FFF7C2FF174802F18C01FFF7BDFF1648DA
:1030500002F1A801FFF7B8FF144802F1C401FFF71D
:10306000B3FF134802F1E001FFF7AEFF114802F190
:10307000FC01FFF7A9FF104802F58C71FFF7A4FFD0
:10308000BDE8084000F0DCB8003802400000024013
:10309000603700080004024000080240000C0240B3
:1030A000001002400014024000180240001C0240C0
:1030B00000200240002402400028024008B500F031
:1030C00033FAFFF7EFFEFEF7FFFFBDE80840FEF71B
:1030D000DBBD000070470000064A536823F001037F
:1030E0005360EFF30983683383F30988002383F384
:1030F0001188704730EF00E010B5202383F311886A
:10310000104B5B6813F4006318D0F1EE103AEFF344
:1031100009844FF0807344F84C3C0B4BDB6844F857
:10312000083CA4F1680383F30988FEF70DFC18B18D
:10313000064B44F8503C10BD054BFAE783F3118869
:1031400010BD00BF00ED00E030EF00E051030008CB
:10315000540300084FF0804310B51A69920708D550
:1031600000241C61202383F31188FFF7DFFE84F322
:103170001188BDE81040FFF7BFBF0000104B1A6C6C
:1031800042F001021A641A6E42F001021A660D4AF8
:103190001B6E936843F0010393604FF080436B22F2
:1031A0009A624FF0FF32DA6200229A615A63DA6063
:1031B0005A6001225A6108211A601C20FFF77ABC6C
:1031C00000380240002004E01B4B1A696FEA4252AB
:1031D0006FEA52521A611A69C2F30A021A614FF079
:1031E000FF301A695A69586100215A6959615A6950
:1031F0001A6A62F080521A621A6A02F080521A62E7
:103200001A6A5A6A58625A6A59625A6A0B4A1068AC
:1032100040F480701060186F00F44070B0F5007FCB
:103220001EBF4FF4803018671967536823F400738A
:10323000536000F059B900BF0038024000700040F0
:10324000354B364A1A64364A4FF4404111601A68C9
:1032500042F001021A601A689207FCD59A6822F0BF
:1032600003029A602C4B19469A6812F00C02FBD1AB
:10327000186800F0F90018609A601A6842F4803209
:103280001A600B689B03FCD54B6F43F001034B673F
:10329000214B5A6F9007FCD5224A5A601A6842F0B7
:1032A00080721A601E4B1A4659684904FCD5196889
:1032B00041F4803119605368D803FCD5136843F496
:1032C00000331360164A53689903FCD5124B1A68F1
:1032D0009201FCD5144A9A6040F20112C3F88C2086
:1032E0000022C3F89020114A40F2073111609A6819
:1032F00042F002029A60084B9A6802F00C02082A17
:10330000FAD15A6C42F480425A645A6E42F48042B6
:103310005A665B6E704700BF003802400004001020
:1033200000700040086C400900948838003C02405E
:10333000084A08B5536911680B4003F00103536153
:1033400023B1054A13680BB150689847BDE808409F
:10335000FFF7D2BE003C0140B0250220084A08B564
:10336000536911680B4003F00203536123B1054A0E
:1033700093680BB1D0689847BDE80840FFF7BCBE22
:10338000003C0140B0250220084A08B55369116885
:103390000B4003F00403536123B1054A13690BB1D9
:1033A00050699847BDE80840FFF7A6BE003C0140C1
:1033B000B0250220084A08B5536911680B4003F094
:1033C0000803536123B1054A93690BB1D06998474B
:1033D000BDE80840FFF790BE003C0140B025022048
:1033E000084A08B5536911680B4003F01003536194
:1033F00023B1054A136A0BB1506A9847BDE80840EB
:10340000FFF77ABE003C0140B0250220174B10B5F3
:103410005C691A68144004F478725A61A30604D5F2
:10342000134A936A0BB1D06A9847600604D5104AD4
:10343000136B0BB1506B9847210604D50C4A936B64
:103440000BB1D06B9847E20504D5094A136C0BB158
:10345000506C9847A30504D5054A936C0BB1D06C0A
:103460009847BDE81040FFF747BE00BF003C014051
:10347000B02502201A4B10B55C691A68144004F498
:103480007C425A61620504D5164A136D0BB1506D2A
:103490009847230504D5134A936D0BB1D06D984717
:1034A000E00404D50F4A136E0BB1506E9847A10487
:1034B00004D50C4A936E0BB1D06E9847620404D5C4
:1034C000084A136F0BB1506F9847230404D5054A7F
:1034D000936F0BB1D06F9847BDE81040FFF70CBE5B
:1034E000003C0140B0250220062108B50846FFF740
:1034F000E1FA06210720FFF7DDFA06210820FFF791
:10350000D9FA06210920FFF7D5FA06210A20FFF78C
:10351000D1FA06211720FFF7CDFA06212820BDE8B1
:103520000840FFF7C7BA000008B5FFF74DFEFDF7EA
:1035300023FDFDF7D1FEFDF7A5FDFFF7CBFDBDE8AF
:103540000840FFF799BC0000034611F8012B03F86F
:10355000012B002AF9D1704712101213121100002A
:103560000010410001105A0053544D3332463F3F82
:103570003F3F3F3F0053544D333246375B347C3539
:103580005D780053544D333246375B367C375D7877
:103590000000000000000000FD0F0008E90F000817
:1035A00025100008111000081D100008091000085F
:1035B000F50F0008E10F000881100008000000006E
:1035C00001000000000000000200000000000000F8
:1035D000291200089112000840004000082B022028
:1035E000182B022002000000000000000300000071
:1035F00000000000D51200080000000010000000CC
:10360000282B022000000000010000000000000044
:10361000CC2D0220010102004172647550696C6F6B
:10362000740025424F415244252D424C00255345FC
:103630005249414C25000000291C0008911B00083C
:10364000951100080D1C00084300000050360008CA
:1036500009024300020100C0320904000001020215
:1036600001000524001001052401000104240202C8
:103670000524060001070582030800FF0904010074
:10368000020A000000070501024000000705810250
:1036900040000000120000009C36000812011001DA
:1036A000020000400912415700020102030100001C
:1036B0000403090425424F41524425005239506900
:1036C0006C6F74003031323334353637383941421B
:1036D00043444546000000000080000000800000D8
:1036E00000800000008000000000020000000400D4
:1036F00000000400000004000000040000000400BA
:103700000000040000000400000000002D14000868
:103710000D170008B917000840004000442E022091
:10372000442E022001000000542E022080000000E0
:1037300040010000050000006D61696E000000009E
:1037400058370008602E0220583002200100000087
:10375000A12E00080000000069646C6500000000F4
:103760000000802A00000000AAAAAAAA0000000007
:10377000FFFF00000000000000A00A0000000000A1
:1037800000000000AAAAAAAA00000000FFFF000093
:103790000000000000000000000000000000000029
:1037A000AAAAAAAA00000000FFFF00000000000073
:1037B000000000000000000000000000AAAAAAAA61
:1037C00000000000FFFF00000000000000000000FB
:1037D0000100000000000000AAAAAAAA0000000040
:1037E000FEFF0000000000000000000000000000DC
:1037F00000000000AAAAAAAA00000000FFFF000023
:1038000000000000000000000000000000000000B8
:10381000AAAAAAAA00000000FFFF00000000000002
:10382000000000000000000000000000AAAAAAAAF0
:1038300000000000FFFF000000000000000000008A
:103840000000000000000000AAAAAAAA00000000D0
:10385000FFFF00000000000000000000000000006A
:103860000000000000000000000000000000000058
:103870000000000000000000000000000000000048
:103880000000000000000000000000000000000038
:103890000000000000000000FF0000000000000029
:1038A000683500083F000000490400007535000835
:1038B0003F00000051040000833500083F00000075
:1038C000009600000000080004000000B036000868
:1038D00000000000000000000000000000000000E8
:0838E0000000000000000000E0
:00000001FF
